:020000040000FA
:040000008A01D22877
:0800080083120313BB20BB208F
:1000100081010B11A00A0F302002031D5628831204
:100020000313860AA001A10AC7308D2130302107B1
:10003000C02099210A302102031D5628A101A20ADD
:10004000C6308D2130302207C92099210630220286
:10005000031D5628A201A30AC4308D213030230786
:10006000C02099210A302302031D5628A301A40AA7
:10007000C3308D2130302407C92099210630240255
:10008000031D5628A401A50AC1308D213030250753
:10009000C02099210A302502031D5628A501A60A71
:1000A000C0308D2130302607992156288B16090043
:1000B000A001A101A201A301A401A501A6010800BC
:1000C00004302502031D080002302602031D08002B
:1000D0005820562108000730C50026308400C50B83
:1000E0007328051008000008C4001D3084070008AC
:1000F000C402031D08001D30840284036F280730EA
:10010000C50026308400C50B8728051008000008AC
:10011000C4002D3084070008C402031D08002D30E0
:100120008402840383280730C50026308400C50B71
:100130009B28051408000008C40017308407000835
:10014000C402031D08001730840284039728073077
:10015000C50026308400C50BAF2805140800000830
:10016000C400273084070008C402031D080027309C
:1001700084028403AB28BB30A800A80BBD2808006C
:10018000A7003A302702031DC7283030080027088F
:100190000800A70036302702031DD02830300800A1
:1001A00027080800831203139813831603130730DC
:1001B0009C009D019B01850186018312031386012A
:1001C00005108312031338308D2101308D21033047
:1001D0008D210F308D2180308D21792221308400B6
:1001E0005621B521B5211922383084005621B52178
:1001F000B5218316031338308400003083120317AF
:100200008D00212383120313492248308400562194
:10021000B521B521831603134830840010308312B2
:1002200003178D0021238312031383120313B921B3
:100230003E3084005621B521B521831603133E308C
:1002400084000730831203178D00212383120313C8
:1002500083120313E9214E3084005621B521B521C4
:10026000831603134E3084001730831203178D005A
:10027000212383120313831203138221213084006C
:1002800056210730831603138100831203130510D0
:100290008601003081008B178B16860160208B123F
:1002A0009320A7206B207F208B164E29C7308D21ED
:1002B000303000079921C6308D21840A3030000784
:1002C0009921C5308D213A309921C4308D21840A7D
:1002D000303000079921C3308D21840A3030000767
:1002E0009921C2308D213A309921C1308D21840A63
:1002F000303000079921C0308D21840A303000074A
:100300009921080080308D21483099214F30992162
:10031000523099214130992108008600A521051508
:100320008510A52105118510A52105158510A5218C
:1003300008008600A52105158514A5210511851441
:10034000A52105158514A52108002330AA00A900C0
:10035000A90BA829AA0BA7290800FA30AA00A9000E
:10036000A90BB029AA0BAF290800AD21AD21AD2101
:1003700008008312031338308D2101308D210330A2
:100380008D210F308D2180308D21443099214530D1
:10039000992153309921313099213A309921C03037
:1003A0008D210630B700433084009D22C500463CB5
:1003B000031DE7294508831603133E3084000730E8
:1003C000831203178D002F2383120313080045089F
:1003D00008008312031338308D2101308D21033042
:1003E0008D210F308D2180308D2144309921453071
:1003F000992153309921323099213A309921C030D6
:100400008D210630B700533084009D22C500463C44
:10041000031D172A4508831603134E308400173036
:10042000831203178D002F2383120313080045083E
:1004300008008312031338308D2101308D210330E1
:100440008D210F308D2180308D2141309921433015
:10045000992154309921313099213A309921C03075
:100460008D210630B7003D3084009D22C500463CFA
:10047000031D472A450883160313383084000030D3
:10048000831203178D002F238312031308004508DE
:1004900008008312031338308D2101308D21033081
:1004A0008D210F308D2180308D21413099214330B5
:1004B000992154309921323099213A309921C03014
:1004C0008D210630B7004D3084009D22C500463C8A
:1004D000031D772A45088316031348308400103023
:1004E000831203178D002F2383120313080045087E
:1004F00008008312031338308D2101308D21033021
:100500008D210F308D2180308D2153309921453040
:100510009921543099213A309921C0308D210630EB
:10052000B700263084009D22C500463C031D9B2A4F
:100530004508582008004508080003308A00831643
:10054000F030860081138312EF30B0008600043053
:10055000B100B00C30088600A52106080F38B200A3
:10056000B209031DB62AB10BA92AA42A06080F381E
:10057000B600B609031DB62A8316031300308600A1
:1005800083120313B00930080F39B0003208F03974
:10059000B004300886001130B200B20332080023E4
:1005A0003002031DCD2A32088600103032070023A6
:1005B000C500463C031DDE2A4508080045088600A4
:1005C000B00000308316031300308600831203133B
:1005D0003008D03E8000303E99218403B70B9D2A1D
:0405E000B521080039
:10060000820711341234143418342134223424343F
:10061000283441344234443448348134823484347C
:10062000883430343134323433343434353436343D
:100630003734383439344134423443344434453423
:1006400046340630B7000008831203178C003823A5
:10065000840A831203178D0AB70B232B0800063078
:10066000B70047238000840A8D0AB70B312B08009E
:10067000831603178C130C158B1355308D00AA307D
:100680008D008C148C18422B0C118B1708008316CC
:0E06900003178C130C14831203170C080800B8
:00000001FF
